:100000000C9407060C944E060C944E060C94482C47
:100010000C944E060C944E060C944E060C944E0610
:100020000C944E060C944E060C94B4140C9470145C
:100030000C94822A0C944E060C944E060C944E0698
:100040000C944E060C944E060C944E060C944E06E0
:100050000C944E060C94B4100C944E060C944E0660
:100060000C944E060C944E060C944E060C944E06C0
:100070000C944E060C944E060C944E060C944E06B0
:100080000C944E060C944E060C944E060C944E06A0
:100090000C944E060C944E060C944E060C944E0690
:1000A0000C944E060C944E060C944E060000000074
:1000B0000000000000000000000000000000000040
:1000C0007E0F00D4FFFFFFC7000000780000000093
:1000D000000000002A2B28000000000000000000A3
:1000E0000000000000000029000000002C1E342049
:1000F000212224342627252E362D3738271E1F206F
:100100002122232425263333362E37381F040506B3
:100110000708090A0B0C0D0E0F10111213141516F7
:100120001718191A1B1C1D2F3130232D35040506F5
:100130000708090A0B0C0D0E0F10111213141516D7
:100140001718191A1B1C1D2F3130354C00010101E5
:100150000101010101010202020202020202020384
:100160000303030303030304040404040404050554
:100170000505050606060606070707070708080817
:1001800008090909090A0A0A0B0B0B0C0C0C0D0DC6
:100190000D0E0E0E0F0F0F1010111111121213135E
:1001A0001414151516161717181819191A1A1B1BD7
:1001B0001C1D1D1E1E1F2020212222232424252633
:1001C00026272829292A2B2C2D2D2E2F303132326B
:1001D000333435363738393A3B3C3D3E3F40414277
:1001E000434445464748494A4C4D4E4F505153545D
:1001F000555658595A5B5D5E5F6162646566686911
:100200006B6C6D6F7072737577787A7B7D7E808290
:10021000838587888A8C8E8F91939596989A9C9ED9
:10022000A0A2A3A5A7A9ABADAFB1B3B5B7BABCBEE9
:10023000C0C2C4C6C9CBCDCFD1D4D6D8DBDDDFE2B6
:10024000E4E7E9EBEEF0F3F5F8FAFDFFFFAA7F55DE
:100250004000AF0102E3640103E30020001D01330D
:1002600000300025023602300200002A5D13000E25
:100270000015000400090000002A00070017000B09
:100280000008001200000002551C00160011000CAE
:100290000018002C00015504550855035104513035
:1002A0005D280001000100010001000100010000C3
:1002B0000001000100010001000100010000000137
:1002C0000001000100010001000100000001000127
:1002D0000001000100010001000100010001000116
:1002E0000001000100010001002900340032002655
:1002F00002370232020000295D0D001000050024C3
:10030000022B0000003700190006000F001D00142A
:1003100000000001001B000A001A002D004C0029FB
:10032000000100010001003600315D010001000103
:1003300000010001000100010001000000010001B6
:1003400000010001000100010000000100010001A6
:100350000001000100010000000100010001000196
:100360000001000100010001000100010001000185
:1003700000010001002B5DC55C0100005C325D33B3
:100380005D00002D5DC95C4000410042000100009D
:10039000002E5DCA5C3D003E003F00450000002F7E
:1003A0005D43003A003B003C00440001002C5D012D
:1003B0000001000100010001000100010001000135
:1003C0000001000100010000000100010001000126
:1003D0000001000100000001000100010001000116
:1003E0000001000000010001000100010001000106
:1003F00000010001000100010001000100010001F5
:100400000049002F0201004B004E002E00000001A9
:1004100000870020022D0238022202000001002184
:100420000252002F001E02890200003902500051C2
:10043000004F008702230201000100010046000175
:10044000002E020100010001000100010001000175
:100450000001000000010001000100010001000195
:100460000000000100010001000100010001000086
:100470000001000100010001000100010001000174
:100480000001000100010001000100010001000164
:100490000002544A004D0001000000010034025FD8
:1004A00000600061002D000000630038005C005D0A
:1004B000005E00330200005300620059005A005BE6
:1004C000003A030100010001006300360001000151
:1004D0000001000100010001000100010001000015
:1004E0000001000100010001000100010000000105
:1004F00000010001000100010001000000010001F5
:1005000000010001000100010001000100010001E3
:1005100000010001000100010000DA02818FD9F121
:10052000DB40A4A62EAF00A0C000A1C800AED580BD
:10053000A81FD300408D14200000047F3F1F6432A9
:1005400014783C1E65666768696A6B6C6D6E6F70C7
:10055000717273740085868788898A8B8C8D8E8FE3
:10056000909192939400A5A6A7A8A9AAABACADAE12
:10057000AFB0B1B2B3B400C5C6C7C8C9CACBCCCD41
:10058000CECFD0D1D2D3000060616200636400009E
:100590008081820083840000A0A1A200A3A40000A7
:1005A000C0C1C200C3C4000075767700787900002E
:1005B0009596970098990000B5B6B700B8B90000B5
:1005C000D5D6D700D8D9000000AE05010980A10119
:1005D000850319012AB700150126B700950175108A
:1005E0008100C0050C0901A101850419012AA0029E
:1005F000150126A002950175108100C005010906AC
:10060000A101050719E029E71500250195087501E5
:1006100081029501750881010507190029FF150060
:1006200026FF009506750881000508190129059522
:100630000575019102950175039101C009023B0006
:10064000020100A0FA0904000001030101000921D0
:10065000110100012240000705810308000A090476
:1006600001000103000000092111010001223200F4
:100670000705820320000A1201100100000008652E
:1006800032030001000102030104033000000022D4
:1006900003480065006C0069007800200072006566
:1006A00000760033002000350072006F0077007381
:1006B0000000001403790075007300680061006B8E
:1006C000006F0062006F00000004030904000000D6
:1006D0000000003E5B4F5B3E003E6B4F6B3E001CDC
:1006E0003E7C3E1C00183C7E3C18001C577D571C6D
:1006F000001C5E7F5E1C0000183C180000FFE7C372
:10070000E7FF00001824180000FFE7DBE7FF0030D8
:10071000483A060E00262979292600407F0505075C
:1007200000407F05253F005A3CE73C5A007F3E1CB5
:100730001C0800081C1C3E7F0014227F2214005F4E
:100740005F005F5F0006097F017F00006689956A90
:100750000060606060600094A2FFA2940008047EC4
:1007600004080010207E20100008082A1C08000839
:100770001C2A0808001E10101010000C1E0C1E0C65
:100780000030383E383000060E3E0E0600000000F5
:1007900000000000005F00000000070007000014D8
:1007A0007F147F1400242A7F2A1200231308646216
:1007B00000364956205000000807030000001C22A4
:1007C0004100000041221C00002A1C7F1C2A000856
:1007D000083E08080000807030000008080808087B
:1007E000000000606000002010080402003E514933
:1007F000453E0000427F40000072494949460021C1
:1008000041494D33001814127F10002745454539E2
:10081000003C4A4949310041211109070036494944
:10082000493600464949291E000000140000000016
:100830004034000000000814224100141414141461
:10084000000041221408000201590906003E415DE2
:10085000594E007C1211127C007F49494936003EF6
:1008600041414122007F4141413E007F4949494188
:10087000007F09090901003E41415173007F0808CA
:10088000087F0000417F4100002040413F01007F80
:1008900008142241007F40404040007F021C027F3C
:1008A000007F0408107F003E4141413E007F09095E
:1008B0000906003E4151215E007F091929460026A4
:1008C000494949320003017F0103003F4040403F56
:1008D000001F2040201F003F4038403F00631408A5
:1008E0001463000304780403006159494D43000078
:1008F0007F41414100020408102000004141417F36
:1009000000040201020400404040404000FCFE029E
:10091000828282828282C2820202FE0000FEFE0287
:1009200062626262E26262E20202FC0000000000B7
:10093000F030400000000000000000000000000057
:1009400000000000000000000000000000000000A7
:1009500000000080000000000000000040000024B3
:10096000A4A4BCA4242400000024A424243C040443
:10097000000000B8A4A4A4BC00000000FC00FC001F
:10098000444444DC44043C00000000FCFEFE7E7E47
:100990007E7E7E7E3E7EFEFEFE0000FEFEFE9E9E73
:1009A0009E9E1E9E9E1EFEFEFC000000000000009B
:1009B00008364100000000770000000041360800C2
:1009C000000201020402003C2623263C007F7F40F7
:1009D000414141414141414140407F00007F7F40D2
:1009E000404040404140404340407F000000F0FB19
:1009F000FB005060FFFC3C1E0E0CFCF8E8E8E83001
:100A000000000000000200000000000000000000E4
:100A10000002020D0202000000000000000000576A
:100A200050575457105000000097949794F70000C7
:100A3000000000E414F494F700000000FF00FF0041
:100A400038A4A4A53C0000000000007F7F7F7E7ECC
:100A50007E7E7E7E7E7E7F7F7F00007F7F7F7F7FAA
:100A60007F7F7E7F7F7C7F7F7F0000000000000013
:100A70000000000000000000000000000000000076
:100A800000000000000000000000000000FEFE0268
:100A9000626262E2626262C20202FE0000FEFE0266
:100AA00082C2E2F2828282820202FE000000077F9E
:100AB000DF0005037F1F1E3C38181F0F0D0D0D06AC
:100AC0000000000000002020508C5020200000007A
:100AD000000000000000000000808040304080895D
:100AE0000906090900000000001C1212121E101055
:100AF000000000000000000000000000FF00738400
:100B0000E794949467000000000000FEFEFE9E9EA5
:100B10009E1E9E9E9E3EFEFEFE0000FEFEFE7E3E51
:100B20001E0E7E7E7E7EFEFEFE00000000000000A7
:100B300000000000000000000000000000000000B5
:100B4000000000000000000000000000003F7F40A7
:100B5000464646474646464340407F00007F7F402A
:100B60004143474F4141414140403F0000000000A8
:100B70000706010000000000000000000000000067
:100B80000000000000000000000100000000000064
:100B90000004000000000000000000010601000049
:100BA0000000000000000000000000000000000045
:100BB0000008083608080000000000001F000E10A2
:100BC0001C121212120000000000003F7F7F797992
:100BD00079787979797C7F7F7F00007F7F7F7E7C49
:100BE00078707E7E7E7E7F7F3F00000000000000E8
:100BF00000000000000000000000000000000000F5
:100C000000000000000000000000000000001124AF
:100C10001FBECFEFDAE0DEBFCDBF04B603FE27C0B4
:100C20008091280990912909A0912A09B0912B0956
:100C30008730904BA740B04BD1F410922809109206
:100C4000290910922A0910922B0914BE84B7877FB4
:100C500084BF0FB6F894A895809160008861809356
:100C60006000109260000FBEE0E0F8E3099529E013
:100C7000AEEBB1E001C01D92A832B207E1F711E07E
:100C8000A0E0B1E0E8E6FCE502C005900D92AE3BC5
:100C9000B107D9F70E94BD250C94FA2D0C940000E1
:100CA000E8EDF0E080818E7F80831092E200109268
:100CB000DA001092E100A0EEB0E08C9181608C939C
:100CC00080818F77808319BCA7EDB0E08C918E7FF7
:100CD0008C9380818F7E80831092030708952091EA
:100CE000E4003091E50095E6A9012091EC00822F07
:100CF000817020FF06C08091E80080FF06C080E080
:100D000008952091E80022FD1AC0809110078823E1
:100D100089F0853089F08091EB0085FD0FC020912E
:100D2000E4003091E50042175307F9F29150E1F6E3
:100D300084E0089582E0089583E0089581E00895B5
:100D4000EF92FF920F931F93CF937C018B010E9430
:100D50006F06C82F811117C08091E80085FD0BC078
:100D60008091E8008E778093E8000E946F068823C8
:100D700099F3C82F08C0F70181917F018093F1009A
:100D80000150110949F78C2FCF911F910F91FF90BE
:100D9000EF9008958091120787FF13C08091E800BB
:100DA00082FF06C08091E8008B778093E80004C042
:100DB000809110078111F2CF089580911007882348
:100DC000D9F38091E80080FFF8CF8091E8008E771A
:100DD000ECCF982F9093E900242F762F50E08917BD
:100DE00031F07091EC002091ED005091F00021FD68
:100DF00007C09F5F973071F78093E90081E0089505
:100E00003091EB003E7F3093EB003091ED003D7F61
:100E10003093ED003091EB0031603093EB00709334
:100E2000EC002093ED005093F0002091EE0027FDA0
:100E3000E0CF80E00895CF92DF92EF92FF920F9380
:100E40001F93CF93DF93C8EDD0E088818F7E888396
:100E5000E7EDF0E080818160808384E082BF81E003
:100E60008093030788818E7F888302EE10E0F8016B
:100E700010821092DA0081EEC82ED12CF601108279
:100E800088818F77888388818068888388818F7D37
:100E9000888319BC109210071092110710920F0747
:100EA00010920E0790EEE92EF12CF70180818B7FD6
:100EB000808388818160888342E060E080E00E94D6
:100EC000E906F60180818E7F8083F8018081816050
:100ED0008083808188608083F70180818E7F80831A
:100EE000888180618883DF91CF911F910F91FF905E
:100EF000EF90DF90CF900895FC01809118079091BA
:100F0000190786179707A0F06115710529F49091CC
:100F1000E8009E779093E80090E06115710551F428
:100F2000911108C08091E80082FF34C080E00895EC
:100F3000BC01F2CF809110078823C1F18530C1F147
:100F40008091E80083FD30C08091E80082FDEACF07
:100F50008091E80080FFE1CF8091F3002091F200C2
:100F6000382F6115710519F02830310558F091E0DE
:100F70002830310509F090E02091E8002E77209389
:100F8000E800CBCF81918093F100615071092F5F10
:100F90003F4FE7CF80911007882341F0853041F023
:100FA0008091E80083FFBECF81E0089582E008953C
:100FB00083E00895089508958091050708959C01A0
:100FC0004FB7F8948091ED069091EE06A091EF0650
:100FD000B091F0064FBF821B930B089580918F064E
:100FE000882331F010928F0610928E0610928D0693
:100FF0000895809590918C06982390938C0608957F
:1010000010928906109288061092870608958091A2
:1010100086068111109286060895E0ECF1E0919128
:10102000891303C0DF0111971C9291E0E63CF90798
:10103000B1F70895A0ECB1E0EFEF90E02D918217A9
:1010400051F0EF3F19F4211101C0E92F9F5F963055
:10105000A9F7EF3F09F408950E2E000CFF0BE254A0
:10106000FE4F8283089527E0929F800D1124982FD0
:10107000977086958695869525E0829FF0011124CC
:10108000E75AF94F50E040E080E0219130E0092E2E
:1010900002C0369527950A94E2F721703327042E73
:1010A00001C0220F0A94EAF7822B4F5F5F4F453051
:1010B000510559F7089527E0929F800D1124982F2C
:1010C000977041E001C0440F9A95EAF7869586959E
:1010D000869595E0899FF0011124E75AF94F90E039
:1010E00080E070E05191DF0111979B01082E02C052
:1010F000369527950A94E2F7217021952527242318
:1011000025272C9301968530910561F708958091EC
:10111000580690912706981301C008958F5F877035
:10112000FACF20910C0330910D032817390771F085
:1011300090930D0380930C03E091A406F091A50613
:10114000309721F00084F185E02D099408952091D5
:101150000A0330910B032817390771F090930B03A2
:1011600080930A03E091A406F091A506309721F040
:101170000680F781E02D09940895E091A406F0918E
:10118000A506309721F00190F081E02D099480E0D0
:101190000895FA01811101C0FB010994EFEBF6E01B
:1011A000118282818460828308958091BA06982F8B
:1011B0009E7F61F4817082608093BA068091BD0643
:1011C000893718F088E78093BD0608958233B0F31D
:1011D00081708063F1CFAF92BF92DF92EF92FF9266
:1011E0000F931F93CF93DF93082F162FE901E42F5E
:1011F000F0E0E45BFE4F611110C0E4915E2F4E2FD2
:101200004983E8835A83DF91CF911F910F91FF901B
:10121000EF90DF90BF90AF900895E62EF12C4491AF
:10122000D42EE42FF0E026E0829FC00111242FEF9E
:1012300030E0B9010E94612D802F90E0880F991F46
:1012400055E5569FD001579FB00D11248A1B9B0B6B
:10125000982F990F890F5901AE18BF08AE9ED00183
:10126000AF9EB00DBE9EB00D11245B2F189F800164
:101270001124012F11275901A01AB10AAE9E800135
:10128000AF9E100DBE9E100D11245901A81AB10871
:10129000AE9CC001AF9C900DBE9C900D1124892F77
:1012A0009927281B390B2E9FC0012F9F900D3E9F21
:1012B000900D1124E92F62307105A1F050F46115F1
:1012C000710509F49DCF6130710581F0EB2F512F2D
:1012D00097CF6430710569F080F06630710509F4CC
:1012E0008FCFF4CFE42F4B2F592F8ACFE42F412FEC
:1012F00087CFEB2F542F492F83CF4B2F5D2DE12F1D
:101300007FCF9091A00692FF06C0282F2871283029
:10131000F9F4877F846093FF06C0282F2871283155
:10132000F1F4877E84612091A10620FF06C0382F4A
:1013300038713830D9F4877F816021FF06C0282FAB
:1013400028712831D1F4877E816194FD877E0895CC
:10135000282F24712430F9F68B7F8860DCCF282F6A
:101360002471243101F78B7E8861DDCF382F3171F4
:10137000313019F78E7F8860E0CF282F217121311D
:1013800021F78E7E8861E1CFCF93DF93972F70E0B6
:1013900027E0929F600D711D1124FB0136E4839FAD
:1013A000E00DF11D1124EE0FFF1FE35AFD4FC59113
:1013B000D491CE01C238D105B9F1E8F5C133D105D8
:1013C00009F499C050F5C932D10509F48DC0CA326B
:1013D000D10509F497C0C11542E5D40708F0B6C09D
:1013E000C11521E5D20708F024C1C83ED10508F097
:1013F0009DC0C13ED10568F5C83AD10508F089C045
:10140000C53AD10508F0EDC0C130D10511F12097E2
:1014100009F443C02497E8F440C0C533D10509F46A
:101420005CC0C933D105B9F62091A006237089F0BC
:1014300080EE90E00EC0C33ED10591F168F4C03E4D
:10144000D105F9F0C23ED10531F62091A00622FD6A
:1014500020C0DF91CF910895C63ED10561F1C73E0E
:10146000D10581F1C43ED10509F0B5CF2091A10687
:1014700021FFEFCF8091A00684FD0FC087EE90E0A2
:10148000E8CF2091A00620FD01C13091A10630FFD8
:10149000E0CF83EE90E024FFDCCF90E080E0D9CF76
:1014A0002091A00622FDF5C03091A10630FDC0CFED
:1014B00024FFCFCFF2CF2091A00623FFCACF24FD77
:1014C000ECCFDCCF2091A00623FDE6C03091A10631
:1014D00031FFEECF84EE90E0BCCF2091A00625FF37
:1014E000B8CF89E290E0B5CF2091A00625FFB1CF1B
:1014F00085E390E0AECF2091A00626FFAACF8AE236
:1015000090E0A7CF2091A00626FFA3CF81E390E033
:10151000A0CFCF3BD10508F6C85AD0E0CC0FDD1FD5
:10152000C959DE4F88819981946493CFC11530E504
:10153000D30708F062C0C11540E4D40708F059C0D1
:10154000DA95C115DF4108F484CFA7CFC11536E580
:10155000D30718F5C11545E5D40708F080C0C115BB
:1015600084E5D80708F076C09C2F96959695AE0135
:1015700043705527C115D34508F460C021E030E021
:1015800002C0220F331F4A95E2F740E2949FC00148
:101590001124822B932B9A685CCFC1153AE5D307AF
:1015A00078F4C11549E5D40708F063C0C11588E592
:1015B000D80708F472CF9C2F8827806F906A49CF94
:1015C000CE0190568115904208F067CF8D2F8F7114
:1015D0000E94810990E0982F882788279F718C2B83
:1015E00046C0C55AD0E0CC59DE4F888190E0906467
:1015F00030CFCE019F70906A2CCF9E01E4E03695EB
:101600002795EA95E1F723708C2F86958695837050
:1016100030E2839FC0011124922BC37021E030E09F
:1016200002C0220F331FCA95E2F7822B932B9C68CE
:1016300010CF9C2F8827816F906A0BCF21E030E07C
:1016400002C0220F331F4A95E2F740E2949FC00187
:101650001124EBCF9C2F8827846F906AFACE8C2FB1
:101660000E94810990E0982F882788279F719062B7
:10167000F0CE8C2F8F700E94810934E0D695C795EB
:101680003A95E1F7CF709C2F9069E3CE89E390E023
:10169000E0CE82EE90E0DDCE86EE90E0DACEBF9234
:1016A000CF92DF92EF92FF920F931F93CF93DF932E
:1016B0008C01C090C706D090C806E090C906F09093
:1016C000CA068091900690919106A0919206B091E1
:1016D0009306C82AD92AEA2AFB2ACFE1D0E0BC2EF9
:1016E000D701C6010C2E04C0B695A795979587958E
:1016F0000A94D2F780FD0EC0219788F7B12C8B2D6C
:10170000DF91CF911F910F91FF90EF90DF90CF90DD
:10171000BF900895B8018C2F0E94C409019761F30E
:10172000EECFCF93DF93EC010E944F0BBE01DF9110
:10173000CF910C94C4090E94910B292F2F70929580
:101740009F7092509E3078F4E92FF0E0E450F24D13
:101750000C94892D803F19F020F4883E20F481E01C
:101760000895843FE1F380E00895883EC0F3813F0F
:10177000D1F7F5CF822F8695869586950895CF93DC
:10178000DF93C0912309D09124098A30C1F42091BC
:101790001A07CE018D519740622F70E00E94612D93
:1017A000281B822F66E00E94552DC82FC15018F4C7
:1017B000DF91CF91089580E20E94BF0BF7CF8D306B
:1017C000E9F4CD51D74020911A07622F70E0CE0185
:1017D0000E94612D281B822F9E01280F311D21158B
:1017E000324018F080E0D0E0C0E0C80FD11DC35EE9
:1017F000D84FD0932409C0932309DACF96E0FE0195
:10180000ADE1B9E001900D929A95E1F7803E08F4C0
:1018100058C086E0FE0111928A95E9F7C09123092C
:10182000D091240946E050E0BE018DE199E00E948C
:10183000A52D9E012D513740892B41F1C90145E06D
:10184000969587954A95E1F741E050E0BA0102C0CC
:10185000660F771F8A95E2F7CB0160911B077091A5
:101860001C07862B972BB9016B5F7F4FE5E07695C0
:101870006795EA95E1F702C0440F551F6A95E2F7B4
:10188000842B952B90931C0780931B072A5F3F4F57
:1018900040911A07642F70E0C9010E94612D481B16
:1018A000463010F4240F311D211572E0370710F077
:1018B00030E020E0235E384F309324092093230941
:1018C00077CFF6E08F9FB00111246353794F46E044
:1018D00050E0CE010E948F2DA1CFCF93DF93EC017A
:1018E000FE018491811103C0DF91CF9108950E9480
:1018F000BF0B2196F5CFCF92DF92EF92FF920F931D
:101900001F93CF93DF936C017B0164E670E088E75F
:101910000E94AF2AEC0197FD12C010E000E0F60132
:10192000E00FF11F849164E670E00E940B2BEC0144
:10193000892B29F40F5F1F4F0E151F0581F70E9499
:101940008E2BCE01DF91CF911F910F91FF90EF90E1
:10195000DF90CF9008952FB7F8948091ED06909185
:10196000EE06A091EF06B091F0062FBF805A954188
:10197000AF4FBF4F8093F1069093F206A093F3060A
:10198000B093F4068091F506811108C062E070E022
:1019900081E592E00E947B0C892B19F08091F5067D
:1019A000089581E08093F506F9CFCF9384E090E02D
:1019B0000E94B22DC82F81E290E00E94B22D982F94
:1019C0008C2FCF910895CF93DF9300D00F92CDB796
:1019D000DEB790911007943019F589837B836A8371
:1019E00082E08093E9008FEF9091E800815095FDAF
:1019F00006C095ED9A95F1F700008111F5CF809121
:101A0000E80085FF0DC050E040E063E070E0CE01EB
:101A100001960E94A0068091E8008E778093E800EE
:101A20000F900F900F90DF91CF910895BC0184E04B
:101A30000C94E30CBC0183E00C94E30CCF93DF9394
:101A4000EC0181E08093E9008FEF9091E8008150F4
:101A500095FD06C095ED9A95F1F700008111F5CF3F
:101A60008091E80085FF14C050E040E068E070E03D
:101A7000CE010E94A0068091E8008E778093E80056
:101A800088E0FE01A6E0B7E001900D928A95E1F7AB
:101A9000DF91CF910895609110018091BA0680FF87
:101AA00020C080910F0143E0849FC00111248A5B14
:101AB0009D4F539A2BB1277F3BB138605FB7F894A5
:101AC000FC01649FE00DF11D1124BF016817790727
:101AD000D1F45FBF8FE594E00197F1F700C00000FB
:101AE0000895809111019091120123E0829FF001ED
:101AF0001124EA5BFD4F8917A0F611821082128231
:101B00008F5F3396F8CFFC014191CF01E8E03BB9FC
:101B1000000000C047FF2BB9440F000000C000C008
:101B200000C02BB900C0EA9591F7D0CFEF92FF9299
:101B30001F93CF93DF93EC0110E0EE24EA94F12C95
:101B400060911301161770F00E944B0D9A818C81E1
:101B500090FF2AC08F5F8C83DF91CF911F91FF9000
:101B6000EF90089520911101422F410F5527551FE5
:101B7000CA019A01220F331F280F391F2A5B3D4FDC
:101B80004091BD06493708F048E770E0C7010E9460
:101B9000752D962F8C816091BC06199F800D1124A4
:101BA0000E94EB081F5FCCCF8150D5CFEF92FF9200
:101BB0000F931F93CF93DF93EC018C81811109C0A8
:101BC00081E08C831092060392E090930E01809343
:101BD0000D01809111019091120123E0829FF0018B
:101BE0001124EA5BFD4F891768F110E003E0609172
:101BF0001301161768F10E944B0D80910D01209181
:101C00000603280F2093060390910E01980F9093DE
:101C10000E01191654F4022E000C330B40911301DF
:101C20004150550B2417350734F0819580930D01F1
:101C3000813009F41C82DF91CF911F910F91FF90A9
:101C4000EF9008951182108212828F5F3396CBCF6E
:101C5000E12EF12C70E0C7010E94752D2091110139
:101C6000820F482F50E020910603022E000C330B08
:101C7000E216F306D4F020910E01022E000C330B75
:101C80002E153F0594F0809F900111242A5B3D4F53
:101C90004091BD06493708F048E76091BC06809145
:101CA000BB060E94EB081F5FA2CFFA01EE0FFF1FD9
:101CB000E40FF51FEA5BFD4F118210821282F3CF11
:101CC0009091BA0690FF14C09091110120911201D9
:101CD00033E0939FF0011124EA5BFD4F921710F05F
:101CE0000C944B0D8183608342839F5F3396F6CFC4
:101CF00008950F931F93CF93DF9300D00F92CDB72A
:101D0000DEB78C018091070381110AC09E012F5F0D
:101D10003F4F48E76FEF0E94EB088A8180930703EB
:101D2000F8016481613069F08091070340E0662327
:101D300061F040E0623011F44091070380E060E020
:101D400004C06091070340E080E00E94600EF8014B
:101D5000848190E0019663E070E00E94752D848399
:101D60000F900F900F90DF91CF911F910F910895D9
:101D70000F931F93CF93DF9300D00F92CDB7DEB7B1
:101D80008C018091BA0680FF13C04091BD0649378F
:101D900008F048E79E012F5F3F4F6091BC06F801B5
:101DA00084810E94EB084B8169818A810E94600EC8
:101DB000F80184818F5F84830F900F900F90DF91E3
:101DC000CF911F910F91089580914502811111C00B
:101DD0008091D80080618093D8008AE18A95F1F7DC
:101DE00000C09091D900892F817090FF82E080938C
:101DF000450281E090914502913009F080E008951C
:101E0000CF92DF92EF92FF926B017C010E94D50886
:101E1000B701A60188E090E0FF90EF90DF90CF90AF
:101E20000C94D82DAF92BF92CF92DF92EF92FF9297
:101E30000F931F93CF93DF9300D00F92CDB7DEB7F0
:101E4000082FF62E142FE22E8091BA0680FF3FC095
:101E5000E82FE695AE2FB0E0A55BBE4F9C91909326
:101E6000BF068E7F823009F040C0493708F048E74E
:101E70009E012F5F3F4F6F2D802F0E94EB084B81FB
:101E800069818A810E94600E8091BB06801308C020
:101E90008091BC068F1104C08091BD06811729F086
:101EA0008091C10682608093C1060093BB06F092C8
:101EB000BC061093BD06EE2051F06091BA067091F9
:101EC000BB068091BC069091BD060E94000F0F904A
:101ED0000F900F90DF91CF911F910F91FF90EF9096
:101EE000DF90CF90BF90AF900895923019F4009199
:101EF000BB06CACF9530D9F39E3031F6EE508E2F07
:101F00008170D82EE695F0E0E45BFD4FA590B4908B
:101F1000C12CBB2460911301C61618F00E944B0D12
:101F2000B3CF2C2D30E0A29EC001A39E900DB29E97
:101F3000900D112470E00E94612D802FD11016C0E9
:101F4000860F40911101420F532F511D9A01220F0C
:101F5000331F240F351F2A5B3D4F412F193708F0DF
:101F600048E76F2D0E94EB08C394D4CF861BE9CFBE
:101F7000EAEBF6E0438121E1421B08F440E021E076
:101F8000628181810C94120FEAEBF6E0438121E13A
:101F9000420F08F44FEF21E0628181810C94120F0F
:101FA000EAEBF6E0628121E1621B08F460E021E0E7
:101FB000438181810C94120FEAEBF6E0628121E10A
:101FC000620F08F46FEF21E0438181810C94120FBE
:101FD000EAEBF6E0818121E04381628188500C9434
:101FE000120FEAEBF6E0818121E043816281885F94
:101FF0000C94120F8091BE06882319F081508093B3
:10200000BE066091BA067091BB068091BC069091A5
:10201000BD060C94000F8091BE06833018F48F5FCC
:102020008093BE066091BA067091BB068091BC0693
:102030009091BD060C94000FEAEBF6E080818E7F54
:10204000808360817181828193810E94000F0E9450
:10205000CE08EFEBF6E08281816082832FEF80E78C
:1020600092E0215080409040E1F700C000000C94C5
:102070004B0DEAEBF6E083E0808311828FEF8283E1
:1020800088E783831482AFEBB6E012968C911297A7
:10209000836012968C9360817181828193810C940C
:1020A000000F6CEE7EEF90E080E00E94E42D60E097
:1020B00082E090E00E94C62D60E083E090E00E9404
:1020C000C62D1092900610929106109292061092D0
:1020D000930660E084E090E00E94C62D60E081E21B
:1020E00090E00E94C62D60E085E090E00E94C62D41
:1020F00060E086E090E00E94C62D6FEF87E090E000
:102100000E94C62D40E050E0BA0188E090E00E94B5
:10211000D82D60E08DE090E00E94C62D40E050E0B8
:10212000BA0188E190E00E94D82D60E087E190E05C
:102130000E94C62D40E050E0BA018CE190E00E9480
:10214000D82D60E080E290E00E94C62D40E050E093
:10215000BA018FE090E00E94D82D40E050E0BA0133
:1021600083E190E00C94D82D78941F921FB61F92B3
:1021700011248F939F93AF93BF938091ED0690911D
:10218000EE06A091EF06B091F0060196A11DB11DDB
:102190008093ED069093EE06A093EF06B093F006C1
:1021A000BF91AF919F918F911F901FBE1F90189567
:1021B0002FB7F8948091ED069091EE06A091EF066E
:1021C000B091F0062FBF089580918C0690918B06F8
:1021D000892B90918A06892B8093BE0180918F066E
:1021E000882319F10E94D81020918D0630918E0617
:1021F000821B930B8838934110F00E94EE07809168
:10220000BE0190918F06892B8093BE0120E080EC67
:1022100091E0FC013191CF0131112F5FF1E0863C5B
:102220009F07B9F721110E94EE07E091A406F091F3
:10223000A506309731F00280F381E02D8EEB91E01E
:102240000994089510928B0610928A060E94E41059
:1022500090E080E00E94A70890E080E00C94910854
:102260006093C7067093C8068093C9069093CA0608
:102270000C9422110F931F9341E050E060E070E056
:1022800004C0440F551F661F771F8A95D2F7CB01F4
:10229000BA0160957095809590950091C706109150
:1022A000C8062091C9063091CA0660237123822393
:1022B00093231F910F910C94301190918906809572
:1022C000892380938906282F277071F4282F082EE0
:1022D000000C330B9217130639F08595859585957B
:1022E0000E943A110C94000808950F931F9341E047
:1022F00050E060E070E004C0440F551F661F771F78
:102300008A95D2F78091C7069091C806A091C90618
:10231000B091CA068A019B01082B192B2A2B3B2B53
:10232000C901B8011F910F910C9430116093900670
:102330007093910680939206909393060C942211C9
:1023400010928C06E0ECF1E086E0DF011D928A95A8
:10235000E9F70C9422111F93CF93DF93CDB7DEB72B
:10236000AA970FB6F894DEBF0FBECDBF82E197E00B
:102370002091F100FC012193CF01F7E08A319F0702
:10238000B9F780911307833009F46FC0B8F4813036
:1023900009F446C0823009F4B0C08091E80083FFA0
:1023A00087C280911207909113079A3008F080C27B
:1023B000E92FF0E0E65FF14D0C94892D8A3009F4A5
:1023C0008BC08B3009F46EC0893039F780911207C9
:1023D000813219F780911607909117070297E8F656
:1023E0008091E800877F8093E8008091E80082FF79
:1023F00037C09091F3008091F200029729F4809108
:10240000F1008B7F813021F48091F10080930507EA
:102410008091E8008B778093E8000E94CA06BDCFC8
:1024200080911207813A09F0B8CF8091E800877F48
:102430008093E8008091160790911707892B61F42B
:1024400068E086E097E070E00E947C078091E800F9
:102450008B778093E800A1CF60E090E080E0F3CF3D
:10246000809110078111C1CF98CF80911207813AD6
:1024700009F093CF8091160790911707892B09F0E7
:102480008CCF8091E800877F8093E8008091E800FE
:1024900080FFFCCF809136018093F1008091E800AD
:1024A0008E77B9CF80911207813209F076CF809173
:1024B000160790911707892B09F06FCF8091E800DC
:1024C000877F8093E8000E94CA068091140780935A
:1024D00036010E94A01161CF80911207813209F06C
:1024E0005CCF8091E800877F8093E8000E94CA0655
:1024F000809115078093040750CF80911207813A8D
:1025000009F04BCF8091E800877F8093E8008091AD
:10251000E80080FFFCCF80910407BECF803899F09F
:10252000823809F0C5C1809116078F70873008F096
:10253000BFC18093E9008091EB0085FB882780F97B
:102540001092E90006C080910E0790910F0791113B
:1025500082609091E800977F9093E8008093F1006B
:102560001092F1008091E8008E779EC1882309F4D3
:102570008CC1823009F09CC18091140781118FC1F8
:10258000809116078F702FEF280F263008F090C12A
:102590008093E9002091EB0020FF81C1933031F45A
:1025A0008091EB0080628093EB0079C19091EB0009
:1025B00090619093EB0021E030E001C0220F8A95FA
:1025C000EAF72093EA001092EA008091EB0088601D
:1025D000EACF81116DC1109114071F778091E3003C
:1025E0008078812B8093E3008091E800877F80933F
:1025F000E8000E94CA068091E80080FFFCCF80912D
:10260000E30080688093E30082E0111183E080930F
:1026100010074EC18058823008F04AC180911407DB
:10262000909115078C3D23E09207A1F583E08A8302
:102630008AE289834FB7F894DE01139620E03EE0EA
:1026400051E2E32FF0E050935700E49120FF03C0E4
:10265000E295EF703F5FEF708E2F90E0EA30C0F0B0
:10266000C7968D939D932F5F243159F74FBF80916B
:10267000E800877F8093E8006AE270E0CE0101966F
:102680000E947C078091E8008B778093E80010C15E
:10269000C096E7CF4091160750911707292F33278F
:1026A0002330310509F445C078F52130310509F4AE
:1026B0007BC08BE390E0ECE3F6E02230310509F0DB
:1026C000F7C02091E800277F2093E80020911807A9
:1026D000309119078217930708F49C0140E02115F7
:1026E000310509F070C041116EC08091E80082FD93
:1026F000C9CF80911007882329F2853019F2809183
:10270000E80083FFF2CFBECF2132310509F440C08B
:102710002232310509F0CCC04115510509F44EC0F3
:102720004130510509F0C4C082E390E0EAECF5E0E5
:10273000C8CF992781309105D9F0009771F0823088
:102740009105F1F0039709F0B3C0E9E8F6E0E491F0
:102750008E2F90E0E9E8F6E007C0E9ECF6E0E491BE
:102760008E2F90E0E9ECF6E0009709F4A1C0A9CF24
:10277000E3EBF6E0E4918E2F90E0E3EBF6E0F4CFAC
:10278000EFE8F6E0E4918E2F90E0EFE8F6E0ECCF92
:102790004115510571F04130510509F089C089E0BA
:1027A00090E0E7E6F6E08DCF82E190E0E7E7F6E043
:1027B00088CF89E090E0EEE4F6E083CF80E490E01B
:1027C000ECEFF5E07ECF80911007882309F45ACF13
:1027D000853009F457CF8091E80083FD53CF809175
:1027E000E80082FD82CF8091E80080FF78CF909151
:1027F000F3008091F2002115310519F08830910520
:1028000050F041E0089709F040E08091E8008E77B1
:102810008093E80064CF44914093F10031962150B9
:1028200031090196E8CF803809F042C08091E80074
:10283000877F8093E800809111078093F10092CE0A
:10284000811136C010911407123090F58091E80084
:10285000877F8093E800109311070E94CA06112316
:1028600011F084E005C08091E30087FDFACF81E09C
:102870008093100742E061EC81E00E94E90642E2A9
:1028800061EC82E00E94E90613C080911407813058
:1028900079F481E0933009F080E080930F07109283
:1028A000E9008091E800877F8093E8000E94CA06D3
:1028B0008091E80083FF0AC08091E800877F8093C1
:1028C000E8008091EB0080628093EB00AA960FB63F
:1028D000F894DEBF0FBECDBFDF91CF911F91089559
:1028E0001F920F920FB60F9211242F933F934F9385
:1028F0005F936F937F938F939F93AF93BF93CF9388
:10290000DF93EF93FF93D091E900DF708091EC00AB
:10291000C82FC17080FDC0E81092E9008091F000DE
:10292000877F8093F00078940E94AB111092E900A9
:102930008091F00088608093F000CD2BCF70C09321
:10294000E900FF91EF91DF91CF91BF91AF919F91FE
:102950008F917F916F915F914F913F912F910F9048
:102960000FBE0F901F9018951F920F920FB60F92E7
:1029700011242F933F934F935F936F937F938F9384
:102980009F93AF93BF93EF93FF938091E10082FFFA
:1029900009C08091E20082FF05C08091E1008B7F39
:1029A0008093E1008091DA0080FF24C08091D800FC
:1029B00080FF20C08091DA008E7F8093DA008091C2
:1029C000D90080FF9FC080E189BD82E189BD09B443
:1029D00000FEFDCF81E080931007809103078111F5
:1029E00009C00E9450060E941B078091E20084608B
:1029F0008093E2008091E10080FF17C08091E200A7
:102A000080FF13C08091E2008E7F8093E20080916E
:102A1000E20080618093E2008091D8008062809320
:102A2000D80019BC85E0809310078091E10084FFF5
:102A30002DC08091E20084FF29C080E189BD82E140
:102A400089BD89B5982F917080FFFBCF8091D80008
:102A50008F7D8093D8008091E1008F7E8093E1008C
:102A60008091E2008F7E8093E2008091E20081609D
:102A70008093E20080911107882309F449C084E023
:102A8000809310070E94A0110E94BD088091E10070
:102A900083FF27C08091E20083FF23C08091E10083
:102AA000877F8093E10082E08093100710921107E6
:102AB0008091E1008E7F8093E1008091E2008E7F23
:102AC0008093E2008091E20080618093E20042E026
:102AD00060E080E00E94E9068091F00088608093C9
:102AE000F000FF91EF91BF91AF919F918F917F91F6
:102AF0006F915F914F913F912F910F900FBE0F906B
:102B00001F90189519BC109210071092030772CFEE
:102B10008091E30087FD93E090931007B3CF882363
:102B200041F0809590918B06892380938B060C94BD
:102B3000E4100895882339F090918B06982B909398
:102B40008B060C94E4100895882321F00E94F90765
:102B50000C94E4100895882339F090918C06982BFA
:102B600090938C060C94E4100895882309F44BC0CC
:102B7000823871F40E94BD0881FF45C089E30E943C
:102B80001A080E94E41089E30E940D080C94E410D6
:102B9000833859F40E94BD0880FF35C083E50E9448
:102BA0001A080E94E41083E5EFCF843859F40E949C
:102BB000BD0882FF28C087E40E941A080E94E41022
:102BC00087E4E2CF9CEF980F913AF0F290E2980FF1
:102BD000983050F4877091E001C0990F8A95EAF718
:102BE000892F0E94F907D2CF9BE5980F933020F4EC
:102BF00090E080E00C94A708885A873120F490E098
:102C000080E00C949108089580911503909116032B
:102C1000009751F10E94B51580911503909116030C
:102C200091FF03C081EE0E94B5158091150390912C
:102C3000160390FF03C080EE0E94B5158091150326
:102C40009091160392FF03C082EE0E94B515809109
:102C500015039091160393FF03C083EE0E94B515F0
:102C600010921603109215030895CF93C82F88234E
:102C700009F488C08238C1F40E94BD0881FD82C079
:102C800089E30E941A080E94E4102FEF81EE94E07D
:102C9000215080409040E1F700C0000089E30E948D
:102CA0000D08CF910C94E4108338A1F40E94BD0864
:102CB00080FD68C083E50E941A080E94E4102FEF8F
:102CC00081EE94E0215080409040E1F700C0000088
:102CD00083E5E5CF8438A1F40E94BD0882FD52C08F
:102CE00087E40E941A080E94E4102FEF81EE94E01E
:102CF000215080409040E1F700C0000087E4CFCF32
:102D00008CEF8C0F813A68F4E0ECF1E08191C81708
:102D100099F121E0E63CF207C9F78C2F0E941A08CE
:102D2000C0CF80E28C0F883068F4C77021E030E0BB
:102D300001C0220FCA95EAF780918C06822B8093FE
:102D40008C06AFCFEBE5EC0FE33040F4F0E0EC594C
:102D5000FE4F808190E0CF910C94A708C85AC731EC
:102D600088F4EC2FF0E0EE0FFF1FE959FE4F808151
:102D70009181CF910C9491088C2F0E940D080E9494
:102D8000E410CBCFCF91089584E00E949A1585E39B
:102D90000E94351685E30E94B51584E00C948F15CA
:102DA000CF93C82F0E943516C93349F42FEF87EE11
:102DB00093E0215080409040E1F700C000008C2F4C
:102DC000CF910C94B515CF92DF92EF92FF920F93B3
:102DD0001F93CF93DF93EC018AE0C82EFE0184910C
:102DE000882309F481C0813009F03EC03196849176
:102DF000813039F42296FE0184910E94D0162196EA
:102E0000EDCF823031F42296FE0184910E94351676
:102E1000F6CF833031F42296FE0184910E94B515DD
:102E2000EECF843009F05EC02296FE01249190E03E
:102E300080E0FE0131962053330B2A30310548F0F3
:102E40000197E8F2EFE9FFE03197F1F700C00000E9
:102E5000F7CFC89EA001C99E500D1124C901840F4F
:102E6000951F2491EF01E5CFE82FF0E0E453FF4FE9
:102E7000D490082F06950695069510E0F801E454C5
:102E8000FF4FE4908770F12C082E02C0F594E79470
:102E90000A94E2F721E0E222FF2404551F4FF801D3
:102EA000049110E002C0159507958A95E2F701702C
:102EB0001127E114F10419F081EE0E943516011575
:102EC000110519F086EE0E9435168D2D0E94D01640
:102ED000012B19F086EE0E94B515EF2809F48FCF6B
:102EE00081EE9CCFEF018BCFDF91CF911F910F919E
:102EF000FF90EF90DF90CF900895CF93DF93C82F8E
:102F0000809110038823B9F10E9404168091140364
:102F1000E0911303F0E097E0899FE00DF11D11248B
:102F200086E4C89FE00DF11D1124EE0FFF1FE35A48
:102F3000FD4FC591D491D1FF03C081EE0E9435169B
:102F4000D0FF03C080EE0E943516D2FF03C082EE90
:102F50000E943516D3FF03C083EE0E9435168C2FD6
:102F60000E943516D0931603C093150310921003D8
:102F700081E080931703DF91CF91089598E0899FB6
:102F800090011124622B609389060E9475110E94A2
:102F9000D810909388068093870608950F931F9307
:102FA000CF93DF93C42FD22FFC0182818823A1F01D
:102FB00040931F060E94D810909309038093080342
:102FC000C77081E001C0880FCA95EAF7DF91CF9101
:102FD0001F910F910C94AB1510911F06141335C05F
:102FE00080910803909109030E94DF07883C9105B6
:102FF00060F5C0E2CD0F1D17B9F080E2810F883077
:1030000040F4177081E001C0880F1A95EAF70E941A
:10301000A415C83048F481E09D2F977001C0880F37
:103020009A95EAF70E94AB15802F0E94D016C830FF
:1030300098F4D77081E001C0880FDA95EAF7DF9144
:10304000CF911F910F910C94A415C77081E001C01E
:10305000880FCA95EAF7F3CFDF91CF911F910F91B7
:1030600008956091BA06669570E04BE050E082E00A
:1030700091E00E94982D892B19F481E08093C0067D
:103080000E94D8109093B5068093B4068091C10633
:1030900084608093C10608959091BA0690FF3BC06A
:1030A000917081112EC092609093BA068091C106F2
:1030B00081608093C106662351F06091BA067091D9
:1030C000BB068091BC069091BD060E94000F6091E6
:1030D000BA06669570E04BE050E082E091E00E9415
:1030E000982D892BA9F00E94CE0881E08093B70625
:1030F00020E04091BD066091BC068091BB060C9417
:10310000120F893110F09063CFCF880F982BCCCF5E
:103110000E943118EACF089561E00C944C18809118
:10312000BA068695815009F488E161E00C944C1848
:103130008091BA0686958F5F893108F081E061E061
:103140000C944C189091BA0690FF07C0969598176A
:1031500020F0961710F40C9498180C948C184F9239
:103160005F926F927F928F929F92AF92BF92CF9217
:10317000DF92EF92FF920F931F93CF93DF9300D0D4
:1031800000D00F92CDB7DEB77C01FC018381948122
:10319000892B39F01081D180812F8D218F3F09F04B
:1031A000E9C60F900F900F900F900F90DF91CF9185
:1031B0001F910F91FF90EF90DF90CF90BF90AF9055
:1031C0009F908F907F906F905F904F9008950E9496
:1031D0004F0B082F682F89819A810E945B08E12F8D
:1031E000F0E027E0D29EE00DF11D112436E4039FAC
:1031F000E00DF11D1124EE0FFF1FE35AFD4F059165
:103200001491F701808190E090931E0680931D0633
:10321000818190E090931C0680931B0622812223DB
:1032200011F105970CF497C00E94E40E81111BC0A8
:1032300020911A06822F90E0FC01EE0FFF1FE80F8D
:10324000F91FE65EFC4F80911D06808380911B066E
:1032500090911C0665E070E00E94752D81831282BA
:103260002F5F20931A068091180390911903892BE0
:1032700039F00033FDE51F0719F081E08093170353
:1032800080911503909116030817190731F4F7017F
:103290008281811102C00E94041603331105A1F03E
:1032A00008F0A5C00431110508F08BC001311105EB
:1032B00058F40A30110508F05AC00730110520F4FF
:1032C0000430110509F05EC0F7018281882309F4FA
:1032D000FBC080E00E947D170E9404164DE552E07D
:1032E00090E09A0180E0F901659174910617170743
:1032F00009F0DDC090931403809313030E94D8104B
:10330000909312038093110381E0809310038093C4
:103310000F0380918906877009F443CFF7018281FA
:10332000882309F43ECF82E00F900F900F900F900A
:103330000F90DF91CF911F910F91FF90EF90DF9051
:10334000CF90BF90AF909F908F907F906F905F9045
:103350004F900C945D110E94E40E811169CF809111
:103360001B0690911C0605970CF47DCF5DCF0B30AA
:10337000110540F00D30110508F4A6CF0E301105EF
:1033800009F4A2CF033FFCE51F0709F493C108F03D
:103390007BC1083D3CE5130709F486C1093D8CE576
:1033A000180709F499C1073D9CE5190709F0F1C018
:1033B00006E221EE41EE67ED7CE5C7010E94CE17E3
:1033C000A8CF0C31110509F47FCF28F4C801459727
:1033D0000497C0F679CF0C32110509F475CF00338C
:1033E000110509F471CF0A32110561F66DCF0C3267
:1033F000FDE51F0709F418C178F5063332E013071D
:1034000009F462CF80F4053292E0190709F45CCF29
:103410000033E2E01E0709F457CF0D31F1E01F073A
:1034200009F0B0CF51CF0A322DE5120709F484C05C
:1034300008F09FC009328DE5180709F0A3CFF70106
:103440008281882309F474C08091A00682FD6DC03A
:1034500081E90E9435165DCF00339DE51907B9F16A
:1034600088F4F70182810E32FDE51F0709F4EEC0F2
:1034700008F4E2C0882309F48CC081E080930E0335
:103480008BE0E1C002333DE5130709F4E7C008F41F
:103490005FC003339DE5190709F074CFF7018281FE
:1034A000882309F476C06091A0066C60DFC08F5F4E
:1034B0002E5F3F4F873009F016CF9F5F425F5F4F0F
:1034C0009A3009F00ECF25CF10920F0322CFF701CB
:1034D0008281882389F01092170381E00E947D1772
:1034E0000E94041681E00E9475110E94D8109093EA
:1034F0001903809318030DCF81E00E943A11809147
:10350000170381110DC080911803909119030E9437
:10351000DF07883C910520F48BE592E00E94E316DA
:103520001092190310921803F4CE0E94C416F1CE23
:1035300081E90E94B515EDCEF7018281882331F033
:103540008091A00682FDF1CF80E983CF80E9F1CFA1
:10355000F7018281882359F08091A00682FD02C084
:1035600084E477CF83E592E00E94E316D2CE84E430
:10357000E0CFF7018281882361F00E9439108091A9
:10358000BA0681608093BA0686950E948C181092C4
:103590000E03F7019281992309F4FDC410921F06CE
:1035A0000230FCE51F0708F47BC106312CE5120749
:1035B00038F098012A5F3C452930310508F070C188
:1035C0000E94D50C9093A1068093A00600313CE5A3
:1035D000130709F434C108F0C2C008309CE519078C
:1035E00009F423C108F091C00430FCE51F0709F479
:1035F00014C108F077C002303CE5130709F403C199
:1036000003301C4509F405C16091A0061091A10684
:1036100084E090E00E94C62D612F81E290E00E943C
:10362000C62D0E94A01175CEF7018281882309F46E
:10363000B0CF0E941C10ADCF882309F4AACF81E03F
:1036400080930E0382E00E948C18A3CF882309F494
:10365000A0CF81E080930E0386E0F5CFF701828151
:103660006091A006637F882309F493CF6093A0063E
:10367000D090A10684E090E00E94C62D6D2D81E2DD
:1036800090E00E94C62D85CF053FECE51E07F1F0C6
:10369000B8F0063F2CE5120709F07BCF07E225EED4
:1036A00046EE66EF7CE589CE07E225EE45EE68ED55
:1036B0007CE583CE06E221EE40EE63EF7CE57DCE35
:1036C00007E225EE44EE64EF7CE577CE06E221EEDC
:1036D00042EE65EF7CE571CE08E221E045EE69ED52
:1036E0007CE56BCE8091A006806106309CE51907D1
:1036F00009F48CC08091A006886007301C4508F44E
:1037000085C08091A006806281C08091A0068D7FD7
:103710000C30FCE51F0709F479C070F48091A00615
:103720008C600A303CE5130709F470C008F481C0CE
:103730008091A0068E7F6AC08091A006877F0E30A0
:103740009CE5190709F462C08091A0068B7F0F30B9
:103750001C4508F45BC08091A0068F7E57C00B3FCC
:10376000FCE51F0709F45DC030F503313CE51307A4
:1037700009F46DC078F401319CE5190709F463C0C0
:1037800002311C4509F040CF0E94A0118091A00693
:103790008F773CC00531FCE51F0709F460C008F4D1
:1037A00074C08091A10681600A3F1C4509F02CCFAE
:1037B0008093A10629CF0F3F8CE5180709F44BC071
:1037C00088F48091A1068D7F0D3FECE51E0781F303
:1037D0008091A1068E7F0E3F1C4550F38091A1067B
:1037E0008360E6CF01302DE5120709F457C008F4D5
:1037F00042C060E002301D4509F006CF8EE090E047
:103800000E94C62D01CF8091A00681608093A00602
:10381000FBCE8091A0068260F9CF8091A0068460E3
:10382000F5CF8091A1068260C3CF8091A00680640D
:10383000EDCF0E94A0118091A0068068E7CF809113
:10384000A0068F7DE3CF8091A0068F7BDFCF809194
:10385000A006837FDBCF8091A1068C7FA9CF8091CA
:10386000A00682FB992790F921E0922790FB82F92C
:1038700090FB83F9CBCF8091A106982F9095917002
:103880008E7F892B90FB81F993CF0E94A01190919C
:10389000A006892F97FB87F98058B8CF61E0AECF9B
:1038A0000631ECE51E0709F06AC080918C068A7A21
:1038B00091E009F490E090932006811102C089E222
:1038C00001C085E30E941A080E94E41022CD85E31E
:1038D0000E940D08F9CF8091BA0680FF03C00E94B4
:1038E0001C1017CD81608093BA0686950E948C18B3
:1038F00010CD4FE858E168E978E10E94C90809CD88
:1039000048E958E16FE878E1F8CF48EE5FE061EF11
:103910007FE0F3CF41EF5FE068EE7FE0EECF40ED78
:103920005FE06CED7FE0E9CF4CED5FE060ED7FE0C4
:10393000E4CF48EB5FE064EC7FE0DFCF44EC5FE096
:1039400068EB7FE0DACF4AEF5FE06BE070E1D5CF64
:103950004BE050E16AEF7FE0D0CF81E0C7CF64E079
:1039600082E00E94A218D5CC6AE085E0FACF6DE033
:103970008BE0F7CF67E18EE0F4CF88E1B7CF011598
:10398000FCE51F0709F447C00E3D1C4509F45FC064
:10399000F70100811181992309F45CC0C8010E94DC
:1039A0004F0BD82E682FC8010E945B08B8018D2DDF
:1039B0000E94C4098C01882EF701C580C2944FE093
:1039C000C422B280B11010928B0680918906877054
:1039D00099F0BB2089F0812F807F803421F080E234
:1039E000800F883048F082E00E945D118091890646
:1039F0008770AA24A3948111A12C912E92943FE068
:103A00009322FBE0F91508F45CC0E92DF0E0EC5ED0
:103A1000F14D0C94892D0E94A0113FEF84E39CE0AE
:103A2000315080409040E1F700C0000087E797E701
:103A3000909301088093000888E19AE00FB6F8940B
:103A4000A895809360000FBE90936000FFCF0E9406
:103A500051105FCCC8010E943308D82EA7CF212F68
:103A60002F70D22E107F19F0D29420EFD222BB20DB
:103A7000C9F0DD2069F080E2800F883010F08110FD
:103A80000BC080918C06D82AD0928C060E94E4103C
:103A9000802F0E94351615C080918B06D82AD092AF
:103AA0008B06F4CF802F0E94B515DD2051F0005E0B
:103AB000083010F0811043C08D2D0E94F9070E943C
:103AC000E410E92DE850FF0B349710F40E94BD0874
:103AD000AA20A9F08091890680FD11C0F701128209
:103AE0008595859585950E947511C7010E94AF182F
:103AF000809189068595859585950E943A1185E086
:103B0000F701DE01119601900D928A95E1F7898106
:103B10009A810E9433089A81E981F0E027E0929F20
:103B2000E00DF11D112436E4839FE00DF11D1124F9
:103B3000EE0FFF1FE35AFD4F8591949132CBD09445
:103B400080918B06D822D0928B06B9CF312F3F704F
:103B5000D32E107F103219F0D29490EFD922882002
:103B600081F081E0881609F44CC0BB2009F455C0EF
:103B7000CC2059F1F701858180FF8ACF8F70858332
:103B800024C0BB2031F1C11004C080918F068D2963
:103B90001DC091E0C9120FC080918F06D82AD81697
:103BA00009F48FCF0E94D81090938E0680938D06D3
:103BB000D0928F0686CFE5E0CE12E7CF0E94EE07C7
:103BC00080918606D812D09286068D2D0E94AB1564
:103BD00078CFC11006C00E94EE078D2D0E94A4155B
:103BE00070CFF1E0CF1208C080918C068D2109F4CE
:103BF00068CF0E940708EFCF25E0C21609F461CF15
:103C0000EACFBB2029F035E03C1508F45ACFDDCFD0
:103C100084E08C1508F455CFE0CFCC20F1F2F9E325
:103C20008F12A1C12FEF37EE83E02150304080404A
:103C3000E1F700C0000097C1812F869586958370BB
:103C400061F0813009F03DCFC8019370B11002C01E
:103C500090E080E00E94910834CFC8019370B110C9
:103C600002C090E080E00E94A7082BCF812F8370D4
:103C700009F066C0B11025CF802F82958695877098
:103C8000880F880F602F6F70462E512C712C612C7D
:103C9000082E04C0440C551C661C771C0A94D2F7ED
:103CA00040E050E0BA0104FF0FC04FE050E060E098
:103CB00070E004C0440F551F661F771F8A95D2F726
:103CC0004095509560957095812F86958695837067
:103CD000823019F1D8F4009190061091910620914C
:103CE000920630919306813069F04429552966295E
:103CF0007729CB01BA0160237123822393230E9489
:103D00009611DFCE402A512A622A732ACB01BA01CA
:103D10006429752986299729F2CF442955296629CE
:103D2000772900919006109191062091920630918A
:103D30009306CB01BA016027712782279327DFCF33
:103D40008695BB2011F0812F8170882309F4B9CEAC
:103D5000802F829586958770880F880F602F6F70EF
:103D6000462E512C712C612C082E04C0440C551C7D
:103D7000661C771C0A94D2F740E050E0BA0104FFB9
:103D80000FC04FE050E060E070E004C0440F551FEA
:103D9000661F771F8A95D2F740955095609570956C
:103DA000812F869586958370823019F1D8F4009121
:103DB000C7061091C8062091C9063091CA06813005
:103DC00069F04429552966297729CB01BA01602376
:103DD0007123822393230E94301173CE402A512AEB
:103DE000622A732ACB01BA01642975298629972989
:103DF000F2CF44295529662977290091C7061091E9
:103E0000C8062091C9063091CA06CB01BA016027C5
:103E1000712782279327DFCF1F70BB2029F0812FC6
:103E20000E947511802FD2CE802F0E94A415812F61
:103E30000E943A1146CE802F92EF891609F455C0A0
:103E4000981578F0E0EF8E1641F1F1EF8F1609F436
:103E500044C0BB2009F482C0C1101ACE812F8F71DB
:103E600041C023EF821609F445C034EF8312F1CF2D
:103E700080918606BB2009F45DC00E94F9078091FD
:103E800089068770843009F048C00E940008812F9D
:103E90008F710E943A11A12C14CEBB20C9F084E08E
:103EA0008C1508F40ECE1F7161E070E080E090E0A8
:103EB00004C0660F771F881F991F1A95D2F70091CB
:103EC000C7061091C8062091C9063091CA069FCF37
:103ED00095E09C1508F4F5CDE6CF812F8F71BB20BE
:103EE00009F4A6CF0E947511ECCD812F8F71BB20F4
:103EF000C9F39ECF60E070E0CB01BB2009F46BCF2B
:103F00001F7161E070E080E090E004C0660F771FF1
:103F1000881F991F1A95D2F75ECFE4E0EC1508F4DC
:103F2000BACF1F71812F0E94751163E0812F0E940B
:103F3000BE17B1CF90918C06982B90938C06F4E02D
:103F4000FC1540F40E9400080E94070864E0812FDD
:103F50008F71EDCF81E00E945D119DCFCC2039F0B3
:103F6000893309F45FCE802F0E94B515AACD812F29
:103F70008F715ECF85E0DE01119601900D928A95DA
:103F8000E1F7F701228189819A81211120C90E94DC
:103F90003308082F24C90631FCE51F0771F0809112
:103FA0008C068272F801E25CFC45E431F10508F010
:103FB000EFCCE05EF14D0C94892D809120068111AB
:103FC00086CC89E285CC1F93CF93DF938091260620
:103FD000807FA9F480912306882389F08091580678
:103FE000D09127066091210670912206A0912406A7
:103FF000B0912506C62FC72316E0D81304C0DF9161
:10400000CF911F91089590E0109711F0CF3F19F4D0
:1040100001968770F2CF189F9001199F300D1124DF
:10402000F901E85DF94F41814713F2CF4081461312
:10403000EFCF42814111ECCF438154814A1B5B0B8E
:10404000483C510528F7809126068F708061809347
:104050002606F901E35DF94F80818F7080618083CE
:1040600081E296E00E94AF18DF91CF911F910C94EE
:104070008708AF92BF92CF92DF92EF92FF920F9399
:104080001F93CF93DF93CDB7DEB761970FB6F89448
:10409000DEBF0FBECDBF8C0185E0F801DE011D96AD
:1040A00001900D928A95E1F7F80180819181E2807B
:1040B00021E2A22E26E0B22E609124067091250600
:1040C0006115710509F43EC1309121064091220627
:1040D000232F24232F3F09F435C1C380D480F090CF
:1040E0002306F601E61BF70BFF2009F4FBC0209125
:1040F0002606522F507FE83CF10508F0BBC0511155
:1041000078C0FE2C491321C038131FC0E1101DC018
:104110002F70206120932606C5010E94AF18809160
:104120002606F80185838F2D61960FB6F894DEBFC1
:104130000FBECDBFDF91CF911F910F91FF90EF90F8
:10414000DF90CF90BF90AF900895CD2829F0282F11
:1041500029232F3F09F014C120E0F22FF170DF2E48
:1041600020FF3DC0209158064091270656E02413B9
:1041700015C08D879E878D859E850E94910B292F66
:1041800022952F702230F8F0243020F59F70F9F03E
:10419000F8019581907FD9F4D12C1FC030E0529F57
:1041A000F001539FF00D1124E85DF94F61819613E2
:1041B00006C06081861303C06281E61210C02F5FC3
:1041C0003F4F2770D4CF9F7011F0882329F3805E72
:1041D000883010F3C8010E94AF18FD2CA4CFEE2048
:1041E00009F4A1CF80912606816080932606F12CE8
:1041F0009ACF491312C0381310C0E1100EC0F80155
:104200002583C8010E94AF1886E0F801A1E2B6E05C
:1042100001900D928A95E1F786CF8D879E878D85D7
:104220009E850E949B0B882309F1EE20F9F0809176
:104230002606803270F020912106309122063887C0
:104240002F831986DB86CA868C87CE0107960E944B
:10425000AF1886E0F801A1E2B6E001900D928A95D0
:10426000E1F70E94E31FFF24F3945DCFC8010E9491
:10427000AF18F9CF51110AC081E296E00E94AF1841
:1042800086E0F50111928A95E9F7B1CF49130FC085
:1042900038130DC0E1100BC0F8012583C8010E943E
:1042A000AF1886E0F50111928A95E9F73CCF8D872A
:1042B0009E878D859E850E949B0B8823B9F2EE20F8
:1042C000A9F280912606803220F2209121063091B9
:1042D00022063A8329831B82DD82CC828E83CE0123
:1042E0000196B5CFE83CF105E0F6FE2CEE2009F48E
:1042F000BDCF491316C0381314C08091260680FD27
:1043000083CF982F907F09F47FCFF8018583903F6A
:1043100009F477CF982F907F905F8F70892B8583DA
:1043200070CF8D879E878D859E850E949B0B811106
:1043300090CF80912606816080932606C8010E9456
:10434000AF18F1CEEE2009F491CF8D879E878D8531
:104350009E850E949B0BF82E882309F487CF86E068
:10436000F801A1E2B6E001900D928A95E1F7809103
:104370002106909122060E94910B0E94E31FD3CE4A
:1043800021E02E25EACE1F93CF93DF93CDB7DEB782
:1043900067970FB6F894DEBF0FBECDBF4B8B5C8B1B
:1043A0006D8B7E8B8F8B1A8A198A85E0FE0173963E
:1043B000DE011D9601900D928A95E1F70E94D810BA
:1043C0002091870630918806821B930B8838934191
:1043D00020F08091890682FF7FC00E94D810209132
:1043E0008D0630918E06821B930B8838934110F016
:1043F0000E94EE0786E0FE013D96DE0117960190D1
:104400000D928A95E1F7CE0107960E943920882304
:1044100089F016E08091580690912706891349C0CB
:1044200067960FB6F894DEBF0FBECDBFDF91CF9178
:104430001F91089586E0FE013796DE0111960190E6
:104440000D928A95E1F78A859B85892B11F38885E2
:104450009F8189238F3FE9F22091270630E0C9012F
:10446000019687709927409158064817190671F4EC
:104470000E94A011109227061092580686E0E1E2F1
:10448000F6E0DF011D928A95E9F7C3CF96E0929F8F
:10449000D001939FB00D1124A85DB94FFE01319654
:1044A00001900D929A95E1F7809327060E94870864
:1044B000B0CF819FC0011124885D994F0E9439209F
:1044C000882309F4ADCF8091580690E0019687705B
:1044D0009927809358069ECF82E00E945D117DCF80
:1044E0002F923F925F926F927F928F929F92AF92A4
:1044F000BF92CF92DF92EF92FF920F931F93CF93D1
:10450000DF93882E962E20910001309101012F3FDC
:10451000320759F58091BA0681608093BA0660E04F
:1045200086950E944C1881E00E948C1880910001B1
:104530009091010101968C3091050CF015C190937A
:10454000010180930001DF91CF911F910F91FF90A6
:10455000EF90DF90CF90BF90AF909F908F907F9023
:104560006F905F903F902F9008952530310508F0AF
:1045700091C05091300250901A06E901CC0FDD1F16
:10458000CE01820F931FDC01A953BE4F3D01FE01F6
:10459000EF5BFE4F1F01551649F2852F90E0DC01BD
:1045A000AA0FBB1FFD01E80FF91FE65EFC4F6181FA
:1045B0008901061B110917FF03C011950195110907
:1045C000E101E880F980F30170E060E0A80FB91F15
:1045D000A65EBC4F6D01D2E0CD0ED11C6E157F05DD
:1045E00014F05F5FD8CF8C915B01A81AB108C501A8
:1045F000B7FE03C0919581959109800F911FE60147
:10460000A880B12CA816B9060CF440C008968A19E7
:104610009B0997FF02C090E080E0880F991F880FE8
:10462000991F009799F1A080DFEFAD1671F08820F7
:1046300061F0A80EB92EB11CCFEFAC16B10421F079
:104640001CF0AA24AA94B12CA082A180DFEFAD16A1
:1046500071F0992061F0A80EB92EB11CCFEFAC1605
:10466000B10421F01CF0AA24AA94B12CA182B2803A
:10467000DFEFBD1659F0442349F08B0D911D8F3F9C
:10468000910519F014F08FEF90E082836F5F7F4FF8
:104690003F96A4CF8091300240911A06982F253082
:1046A000310589F1C90106978530910508F050C0A0
:1046B000EC01CC0FDD1FFE01EF5BFE4F60817181CD
:1046C000FE01E80FF91FE953FE4F30E020E0C95C1E
:1046D000DE4F817099278B0101501109261737078A
:1046E000CCF00E944B0D22CF292F30E0F901EE0FC4
:1046F000FF1FE20FF31FE65EFC4F2281223140F4E0
:104700002F5F22839F5F4913EFCF809330020ECF3C
:104710008F5FF8CFA881B981A801421B530B009786
:1047200009F0A9014A0F5B1FDA01AA0FBB1FA40FF2
:10473000B51FAA5BBD4F408111964C9311974181E3
:104740004C93428112964C932F5F3F4F3F96C6CFBA
:104750002B30310509F0EACEE7ECF1E089E6DF0124
:104760001D928A95E9F7E2CE1092010110920001A4
:10477000EACE8F929F92AF92BF92CF92DF92EF924A
:10478000FF920F931F93CF93DF9365E971E004E9E4
:1047900016E04801C0E0CC24C394D12CDB018D91FC
:1047A000BD01E82FE295EF70F0E091A18F707601E6
:1047B00001C0EE0C8A95EAF7892F8E2981A382A188
:1047C000DE2DD0958D2382A3B0EABA95F1F78FE95B
:1047D000A82E81E0B82E50E040E020E0D5013D91C8
:1047E0005D01832F82958F7090E0DC0190968C9113
:1047F00090E03F7002C0959587953A95E2F780FD6D
:1048000045C08C2D042E01C0880F0A94EAF7282B8E
:104810004F5F5F4F4730510509F781A18D2381A379
:1048200082A1E82AE2A2F4018081281789F120837D
:1048300081E0C82BFFEF8F1A9F0A21E06A397207C7
:1048400009F0ACCFD0919F06CC2321F181E0809379
:1048500033020E94D81090933202809331028091EB
:104860003102909132020E94DF070697B8F0ED2FD7
:10487000F0E0E955F94FD8018D918D018193B6E0B3
:1048800009391B07C1F71092330208C080E0BFCF7F
:1048900080E0CFCF809133028111E1CF0E94E40EFE
:1048A000882309F4FFC0D0919E068091C106882319
:1048B000E9F085E0EAEBF6E0A5E3B2E001900D92C5
:1048C0008A95E1F78091BF069091C006A091C1063C
:1048D00080933A0290933B02A0933C0281E090E0E7
:1048E0000E94D72C892B11F41092C10690E080E031
:1048F0000E94D72C009709F46EC0809144028F5F0C
:1049000080934402863008F092C08091100388237F
:1049100091F080911103909112030E94DF078C3473
:10492000910548F080E00E947D1780910F0381116E
:1049300002C00E9404168091C7069091C806A091FB
:10494000C906B091CA064091340250E070E060E0C0
:10495000481759076A077B0789F084309105A1053C
:10496000B10509F483C008F06DC00297A105B10537
:1049700009F474C08091C7068093340280910E03BD
:1049800081111BC08091C7069091C806A091C906ED
:10499000B091CA0684309105A105B10509F47FC024
:1049A00008F066C00097A105B10509F46FC044E6A0
:1049B0000297A105B10509F473C08C2FDF91CF9147
:1049C0001F910F91FF90EF90DF90CF90BF90AF902D
:1049D0009F908F900895ED2FF0E0E955F94FDC019D
:1049E000A25CBD4F2C912193019685309105B9F7BA
:1049F000E091A306F0E0EE53F94F809143029081DD
:104A0000891B982F04C0915020812F5F2083191695
:104A1000D4F3982F87FD90E0891B811103C0109279
:104A2000440273CF8F5F908191509083F6CFE091D5
:104A30009E06F0E0E955F94F10821182128213822E
:104A4000148263CF88309105A105B10569F04097C4
:104A5000A105B10509F08ECF84E001C081E00E947C
:104A60007D170E94041686CF83E0F9CF82E0F7CF4E
:104A700088309105A105B10579F040E067E14097E4
:104A8000A105B10509F099CF8FE703C04FE760E7B3
:104A900080E00E94702291CF40E06FE7F9CF4DE3B4
:104AA00060E0F2CFE0919F060E2F10E080913D0272
:104AB000883099F580913C0280FF0FC090913502BB
:104AC0008091BA0690FF40C081608093BA068091C1
:104AD000350260E086950E944C1880913C0281FF6F
:104AE00009C020E04091380260913702809136027F
:104AF0000E94120F80913C0282FF06C080913B020F
:104B00008823C1F10E94311880913C0283FF03C0C9
:104B100081E08093B70610923D02F801E955F94F04
:104B200090E080E02191DC01A25CBD4F2C930196C6
:104B300085309105B9F7E091C506F0E0EE53F94FE5
:104B400080818093430239CF8E7F8093BA060E9482
:104B5000CE088091C10681608093C106EFEFF0E737
:104B600022E0E150F0402040E1F700C000000E9448
:104B70004B0DB3CF0E94CE08C7CFCDB7DEB72D9770
:104B80000FB6F894DEBF0FBECDBF84B7877F84BF5A
:104B90000FB6F894A89580916000886180936000BA
:104BA000109260000FBE80E890E00FB6F8948093FA
:104BB0006100909361000FBE85B7806885BF85B79F
:104BC000806885BF0E9450060E941B078091E2000A
:104BD00084608093E2007894809110078823A1F08C
:104BE0001091E9001F709091EC00892F817090FD69
:104BF00080E8182B1092E9008091E80083FD0E9464
:104C0000AB111F701093E90082E084BD93E095BD65
:104C10009AEF97BD80936E0022982A9A579A5F98D0
:104C200025E02A95F1F7000083B182FB882780F9FF
:104C300057985F9A30EA3A95F1F780932401809172
:104C40002401882309F440C310920F0180E280936D
:104C500010010E94E40E882331F062E070E084E1EC
:104C600091E00E94F52B809124018091240195E030
:104C7000811190E090939F0685E0891B80939E06AA
:104C8000A5E9B1E02AE931E041E050E08D91E82F5B
:104C9000E295EF70F0E011A18F70BA0101C0660FCC
:104CA0008A95EAF7962F9095912391A382A1862B5E
:104CB00082A32A173B0751F7AFE9B1E026EA31E0BA
:104CC00041E050E08D91E82FE295EF70F0E011A106
:104CD0008F70BA0101C0660F8A95EAF7962F9095FA
:104CE000912391A382A1862B82A32A173B0751F718
:104CF000E4E9F6E08EE996E0A7EAB6E011921D92AB
:104D00008E179F07D9F790E080E00E94C02D8C3E5F
:104D10009E4F11F00E9451100E94E40E811106C0B6
:104D200062E070E084E191E00E94FE2B1092EB06BD
:104D300080E880931A070E94A92A6DE070E08CE257
:104D400095E00E947B0C892B09F046C08091EB0610
:104D500063E070E081FDBCC289E295E00E947B0CBB
:104D6000892BD1F56DE070E089E195E00E947B0C24
:104D7000892B91F52FB7F8948091ED069091EE066E
:104D8000A091EF06B091F0062FBF805A9541AF4F2A
:104D9000BF4F8093F1069093F206A093F306B09371
:104DA000F406EDE1F7E080E092E0DF019C011D9266
:104DB00021503040E1F7F0932409E09323098FEF6D
:104DC0009FEF90931C0780931B0781E08093F6066A
:104DD0008093F5061092EC0690E080E00E94C02DD2
:104DE0008C3E9E4F11F00E94511082E090E00E9494
:104DF000B22D8093F8060E94D50C9093A106809363
:104E0000A00683E090E00E94B22D682F70E090E051
:104E100080E00E9496118091A20681113BC090E033
:104E200080E00E94C02D8C3E9E4F21F00E945110C8
:104E30000E94391088E090E00E94BA2D6093BA0673
:104E40007093BB068093BC069093BD068091C1060B
:104E500083608093C1066E7F71F40E94391088E0F0
:104E600090E00E94BA2D6093BA067093BB068093BF
:104E7000BC069093BD060E94D5080E94CE08809182
:104E8000BA0680FF04C060E086950E944C1881E05D
:104E90008093A20626982E9A25982D9A83B186FB98
:104EA000882780F91D9917C290E0892B8093C60648
:104EB0009091240181E098279093C506891B8093E7
:104EC000A3068CE291E09093A5068093A4065DE191
:104ED000652E57E0752E44244394512C8091100781
:104EE000853009F4FAC10E94B923D82E0E94E40E3D
:104EF000882309F437C2E9EFF6E0A7EAB6E010E04C
:104F000000E0302F8D919191981709F425C2292F37
:104F1000282790E0FF24F3944F2D422309F417C271
:104F200099833A838F2191E009F490E09B830E945A
:104F3000D8108160782F9D838C8349815A816B8141
:104F40008D810E94C321F801E750F94F8081F82636
:104F5000F0828091C006882309F46AC08091BF0660
:104F6000E091BA06E695E81BE093B606823009F0B8
:104F70000AC2F0E0EF5BFA4FE4910E2F10E048EB2D
:104F8000E42E4EE0F42E8091B706882389F010922B
:104F9000B7060E94D810980120953095820F931F74
:104FA0009093B5068093B4061092B9061092B80695
:104FB0008091B4069091B5060E94DF078017910793
:104FC000B8F18091B3068823B1F01092B3068091B6
:104FD000B1069091B2060E94DF078033954758F0E2
:104FE0000E94D8109093B2068093B1068091C106BA
:104FF00088608093C106A090B806B090B906E09191
:10500000B406F091B5060E0F1F1F1093B50600935E
:10501000B40684EB96E0F70109958091B80690916B
:10502000B906892B29F4AB2819F081E08093B306E7
:10503000E091C606EE0FEE0FE093C60683B186FB45
:10504000222420F81D99CCC180E08229E82BE0932E
:10505000C6069091C506EF70F0E0EA55FE4F8081DC
:105060002091C406820F84300CF4BDC1E92F990F42
:10507000FF0BEE53F94F90819F5F9083837887FFFA
:1050800003C081508C6F8F5F8093C4068091F606B9
:10509000882309F40AC170922409609223090E94AE
:1050A000BD08B12CA12C80FF03C0B4E0AB2EB12C05
:1050B0000E94BD08F12CE12C81FF03C0A4E0EA2E80
:1050C000F12C0E94BD0810E000E082FF02C004E065
:1050D00010E08091C7069091C806A091C906B091D2
:1050E000CA06F4E08F2E912C0497A105B10511F0AA
:1050F000912C812C53E0AA0CBB1C5A95E1F7C501F9
:1051000088579A4F0E946D0C63E0880C991C6A9531
:10511000E1F7C40184579A4F0E946D0C84E495E036
:105120000E946D0CC50180579A4F0E946D0CC401FE
:105130008C569A4F0E946D0C85E595E00E946D0C8F
:10514000F2E0EF0EF11C73E0EE0CFF1C7A95E1F734
:10515000C70188579A4F0E946D0C0E5F1F4FE3E006
:10516000000F111FEA95E1F7C80184579A4F0E947A
:105170006D0C86E695E00E946D0CC70180579A4F32
:105180000E946D0CC8018C569A4F0E946D0C87E7E7
:1051900095E00E946D0C20911B0730911C07211592
:1051A000310509F457C08091EC06811153C0082FD6
:1051B00010E07201082E02C0EE0CFF1C0A94E2F708
:1051C000A9014E215F21452B09F418C19091EB06EE
:1051D00090FD16C18295880F8076809327019801F3
:1051E000369527953695279520932A01815E8093E1
:1051F000280110922B0124E630E047E050E065E200
:1052000071E088E70E943A2B892B21F5A80195E0EF
:10521000440F551F9A95E1F78091EB0680FDFEC083
:10522000435E584F04E610E020E230E060E488E797
:105230000E94612B892B71F40E94AB0CE094F094D6
:1052400080911B0790911C07E822F922F0921C071D
:10525000E0921B078091F506882339F12FB7F89467
:105260008091ED069091EE06A091EF06B091F006C8
:105270002FBF4091F1065091F2066091F3067091B4
:10528000F406841B950BA60BB70BB7FD0EC08091DF
:10529000F506882351F062E070E088EC95E00E940A
:1052A0007B0C892B11F41092F506D1100E94AB0CE7
:1052B0000E94BD089091F706891709F40FCE0E944D
:1052C000BD088093F7060ACE80E280930F01BFCC21
:1052D00086E295E043CD92E0E8CD809110078430DE
:1052E00021F11092A60688E190E020E40FB6F89430
:1052F000A895809360000FBE2093600083B7817FE4
:10530000846083BF83B7816083BF7894889583B7B7
:105310008E7F83BF0FB6F894A89580916000886156
:1053200080936000109260000FBE80910F07882369
:1053300009F4D4CD0E94B92381EB96E0E7EAF6E0C8
:1053400021912111C9C08E179F07D1F7C7CD9F5F4B
:10535000FF0C973009F0E0CD0F5F1F4F0A301105A9
:1053600009F0CFCD8FEF8E838F8318860E94D810DF
:105370008160782F9A8789874E815F8168858A85C9
:105380000E94C321E6CD853061F4E695F0E0E25C51
:10539000FA4FE4910E2F10E036E9E32E3DE0F32EB4
:1053A000F2CD8B3059F4F0E0E55CFA4FE4910E2F2A
:1053B00010E026EDE22E2DE0F22EE5CD883149F405
:1053C000E9E3F5E00591149199E7E92E9EE0F92EC5
:1053D000DACD00ED17E08AEDE82E87E0F82ED3CD88
:1053E00082E090E032CE8D3F0CF048CEE92F990F4D
:1053F000FF0BEE53F94F908191503FCE8F5FD7CE88
:10540000880F880F880F8093270110922A01895FE7
:105410008093280183E080932B01EDCE80E2ABECFA
:10542000B6E01D928A95E9F70AEB11E0E6EBF1E0B0
:10543000FC87EB87D801ED918D01AB85BC856D9123
:10544000BC87AB87640F752F711D635E784FF0E0EA
:10545000E553F94F30E020E087E0982E921AC42CF3
:10546000022E01C0CC0C0A94EAF75B0190E0D50152
:105470008D915D018C21A92DA91BA770AD870A2EE6
:10548000000CBB0B882E0D8401C0880C0A94EAF72F
:105490008D86B195A195B109A770BB2701C08695EE
:1054A000AA95EAF7882A8081882A80829F5F9830AF
:1054B000F1F62F5F3F4F31962830310569F62EEB1C
:1054C00031E02017310709F0B5CF04E610E020E203
:1054D00030E04BEC56E0AACE80E189BD82E189BD87
:1054E00009B400FEFDCF8091D8008F7D8093D80055
:1054F0008091E00082608093E0008091E00081FD77
:10550000FCCFECCC1F921FB61F9211248F939F9358
:10551000AF93BF938091A606811113C08091ED06D1
:105520009091EE06A091EF06B091F0064196A11D74
:10553000B11D8093ED069093EE06A093EF06B09315
:10554000F006BF91AF919F918F911F901FBE1F904A
:1055500018951092B9008CE08093B8000895EF92EE
:10556000FF920F931F93CF93DF93182FEB011092AD
:10557000BC0084EA8093BC000E94D8107C0180911A
:10558000BC0087FF27C08091B900887F883029F050
:105590008091B900887F8031D9F51093BB0084E8F1
:1055A0008093BC000E94D8108C018091BC0087FFC2
:1055B00024C02091B900287F90E080E02831B1F02C
:1055C00081E090E0203411F490E080E091958195A5
:1055D00091090CC0CF3FDC0791F20E94D8108E19C0
:1055E0009F098C179D0758F28EEF9FEFDF91CF91A7
:1055F0001F910F91FF90EF900895CF3FDC07A9F224
:105600000E94D810801B910B8C179D0770F2ECCF75
:105610008FEF9FEFEBCF0F931F93CF93DF93EB01B0
:105620008093BB0084E88093BC000E94D8108C015A
:105630008091BC0087FF11C02091B900287F81E0D4
:1056400090E0283211F490E080E0919581959109E5
:10565000DF91CF911F910F910895CF3FDC0741F368
:105660000E94D810801B910B8C179D0708F38EEFBA
:105670009FEFEECFCF92DF92EF92FF920F931F93A7
:10568000CF93DF936B018A017901B9010E94AF2AA0
:10569000E6010C0D1D1DC017D10761F424E920930C
:1056A000BC00DF91CF911F910F91FF90EF90DF90A1
:1056B000CF90089597FDF2CFB70189910E940B2BEF
:1056C000EACFCF92DF92EF92FF920F931F93CF9387
:1056D000DF93C62F6A017901B8010E94AF2A97FDB6
:1056E0000CC0B8018C2F0E940B2BE601EC0CFD1CAA
:1056F000CE15DF0511F097FF0CC024E92093BC0004
:10570000DF91CF911F910F91FF90EF90DF90CF909D
:105710000895B80189910E940B2BEACF84E9809308
:10572000BC0008958EE14A9B02C08150E1F74A9B7C
:10573000FECF08955A9880E28A95F1F75A9A089513
:10574000FC013BE03A95F1F720E090E080E031E0A9
:1057500040E14A95F1F7880F4A9B02C081602327F8
:1057600042E04A95F1F7000040E14A95F1F79F5F6A
:105770006913EECF90E19A95F1F799B132E03A953D
:10578000F1F7000040E14A95F1F792FB992790F973
:1057900092272081920F90830895EF92FF920F93AA
:1057A0001F93CF93DF930F92CDB7DEB719828C0191
:1057B0007C01E60EF11C0E151F0561F481E0998154
:1057C000911180E00F90DF91CF911F910F91FF9089
:1057D000EF9008950E94922B68E0CE0101960E94FE
:1057E000A02BF80181938F01E6CF90932709809336
:1057F000260960932509529A5A9A08959093270989
:10580000809326096093250952985A9AEA9AE9E604
:10581000F0E080818F7C808308956150770B91E068
:1058200001C0990F6A95EAF720E031E0911108C0B4
:10583000222391F05A9A80E28A95F1F75A980895B6
:10584000492F482339F05A9A232740E24A95F1F725
:105850009695ECCF5A98F9CF5A98EDCFFF920F93C7
:105860001F93CF93DF93EC018C01060F111DC0171E
:10587000D10731F4DF91CF911F910F91FF900895DF
:10588000F9900E949A2B68E08F2D0E940D2CEFCF8B
:105890001F920F920FB60F9211240F931F932F9305
:1058A0003F934F935F936F937F938F939F93AF93A8
:1058B000BF93EF93FF93CF93DF930F92CDB7DEB7F4
:1058C00019820E94922B67E0CE0101960E94A02BC4
:1058D000082F069506950695982F92959570202F7E
:1058E0002570920F292F2370969596958770920FA9
:1058F000891344C08981811141C080912509801795
:10590000E8F120E12A95F1F75A9A529A82E08A95B5
:10591000F1F700C0A8E00A9FC001112400912609F8
:1059200010912709080F191F5A98F80165816623FD
:1059300021F0868197810E942E2C0E949A2BF0E103
:10594000FA95F1F75A9852985A9A20E12A95F1F768
:10595000D80112966C911297662331F113968D91AE
:105960009C910E94CD2BD801ED91FC91882311F0E0
:1059700088E001C082E080830E94922B0F90DF912B
:10598000CF91FF91EF91BF91AF919F918F917F91B7
:105990006F915F914F913F912F911F910F910F90B8
:1059A0000FBE0F901F901895ED91FC91E1CF0F93D2
:1059B0001F93CF93DF9320912509281719060CF424
:1059C00071C08C0193E0000F111F9A95E1F7C0910F
:1059D0002609D0912709C00FD11FF894529A5A98DE
:1059E00025E02A95F1F70000982F9695957085701F
:1059F000980F892F837096959695980F092B0E9482
:105A00009A2B00C067E0802F0E940D2C80E18A95C0
:105A1000F1F752985A9A4A9B17C087E090E04A994A
:105A200015C06D81662321F18E819F810E94CD2B4F
:105A300081111EC0529A5A9AE881F98182E08083CE
:105A4000789482E090E00DC000C0E5CF019771F43A
:105A5000529A5A9AE881F98181E08083789481E0B2
:105A600090E0DF91CF911F910F91089500C0D7CFA3
:105A70000E94922B20E22A95F1F75A98529A80E1DF
:105A80008A95F1F76A81662321F08B819C810E94BF
:105A90002E2C0E949A2BE881F9811082789490E054
:105AA00080E0DFCF84E090E0DCCF991B79E004C098
:105AB000991F961708F0961B881F7A95C9F780954D
:105AC0000895AA1BBB1B51E107C0AA1FBB1FA61745
:105AD000B70710F0A61BB70B881F991F5A95A9F797
:105AE00080959095BC01CD01089597FB072E16F483
:105AF000009407D077FD09D00E94612D07FC05D0E6
:105B00003EF4909581959F4F0895709561957F4FD4
:105B10000895EE0FFF1F0590F491E02D0994FB010D
:105B2000DC0102C005900D9241505040D8F7089515
:105B3000FC014150504030F001900616D1F73197EA
:105B4000CF010895882799270895FB01DC0104C03F
:105B50008D910190801921F441505040C8F7881B65
:105B6000990B0895F999FECF92BD81BDF89A9927B6
:105B700080B50895A6E1B0E044E050E00C94EC2D2F
:105B8000A8E1B0E042E050E00C94EC2D262FF9990A
:105B9000FECF92BD81BDF89A019700B4021639F08C
:105BA0001FBA20BD0FB6F894FA9AF99A0FBE08955D
:105BB0000396272F0E94C72D0E94C62D252F0E94D5
:105BC000C72D242F0C94C72D0196272F0E94C72D77
:105BD0000C94C62DDC01CB01FC01F999FECF06C067
:105BE000F2BDE1BDF89A319600B40D92415050409B
:105BF000B8F70895F894FFCFAA0BAA0BB30BB30B19
:105C0000B50BB30BB30BB30BAA0BAA0BBA0BB30BAD
:105C1000B30BBA0B8E12B6125814B6125814E912FE
:105C20000A135814131420142F1D2F1DA61DA61D72
:105C30001C1E611D611D611D361E0C1F1B1F1B1FBD
:105C40006B1C791C801C851C8A1C8F1C941C991C45
:105C50009E1CA31CA81CAD1C8919AF1CB41C89195F
:085C6000B71C8919BA1CBD1C18
:105C6800F6FF010E0F10111213141516170102007A
:105C780040004040C60100C601063E023D0208350C
:105C880002000000010021007F220003DC071E0D36
:105C9800DB071A0D160D01000006000C0012001992
:105CA80000060006000600070007000001020202C5
:105CB8000505050505050B0B0B0E0E0E0E0E0E0E3B
:105CC8000E0E0E18818283E200E900EA00B500B6E4
:105CD80000B700CD008301CC008A01920194012114
:105CE80002230224022502260227022A02B300B454
:105CF800006F007000946697C6340000000000F43E
:105D0800F5F6F731333200FF0100010000FFFF0014
:0E5D180000010001FF0000081018181008001C
:00000001FF
